:100000003A280F398A0182075534563459345A3404
:100010006534663469346A349534963499349A3444
:10002000A534A634A934AA340F398A0182070034D2
:10003000083404340C3402340A3406340E340134E7
:10004000093405340D3403340B3407340F340F39BD
:100050008A0182076934A934593499345634963464
:100060006634A6346A34AA345A349A3455349534F2
:100070006534A5348312031307309F0083160313DE
:10008000F930850083160313FF30860083120313B3
:100090002130900083120313003085006400831226
:1000A00003138E018F01851D4E28640064300F02FA
:1000B00003194E288519552806300F02031C4E28B7
:1000C0008E018F01640008300F0203194E28851D30
:1000D000622802300F02031C4E288E018F0120304F
:1000E000FF00640002300F0203194E2885197128A1
:1000F0008E018F01640004300F0203194E28851D04
:100100007A2801300F028E018F01A50DA40DA30DD9
:10011000A20DFF0B712822092302031D4E2824097A
:100120002502031D4E2803302205031D4E28220EF2
:1001300014200120FF007F0E831203170F39E038CF
:10014000A2007F0EF039A300831203138030240233
:10015000031DB0280C302205031D4E280030F8285E
:1001600090302402031DBA280C302205031D4E28AE
:100170000130F82888302402031DC4280C302205E1
:10018000031D4E280530F82898302402031DCE2880
:100190000C302205031D4E280430F8288730240532
:1001A000031D4E28030122190838241B0438A41902
:1001B0000238241A0138A219043E2720FF007F0EBE
:1001C000831203170F39A3047F0EF0390438A400FB
:1001D000A5011630A0004030A10011211C30A00064
:1001E0004030A1001121831203130230A41A0330FE
:1001F0000120FF0083120317F030A3057F0E0F3993
:10020000A3047F0EF0390838A400A5011630A00021
:100210004030A10011211C30A0004030A10011216C
:100220004E2864008312031305181A296400051C64
:1002300016291D29640005181A2983120317A21F05
:100240002C29831203137830A00085146400000069
:1002500000008510A00B252983120317220DA90D7C
:10026000A80DA70DA60DA50DA40DA30DA20DA1030C
:10027000A00B11296400220DA90DA80DA70DA60D34
:0E028000A50DA40DA30DA20DA10B3A29080097
:02400E00453F2C
:00000001FF
